** EXPERIMENTAL (HLL) ** Open Watcom Linker Version 1.6beta1 Limited Availability
Portions Copyright (c) 1985-2002 Sybase, Inc. All Rights Reserved.
Created on:       12/01/07 19:00:23
Warning! W1121: file U:/tmp\ldconv__bsddb_obj_ddce4f08029e148440.obj(U:\DEV\python-2.7.2\Modules\_bsddb.c): '_init_bsddb' has already been exported
Executable Image: build/lib.os2knix-2.7/_bsddb.pyd
creating an OS/2 EMX dynamic link library


                        +------------+
                        |   Groups   |
                        +------------+

Group                           Address              Size
=====                           =======              ====

CGROUP                          0001:00000000        000f3590
DGROUP                          0002:00000000        00002350



                        +--------------+
                        |   Segments   |
                        +--------------+

Segment                Class          Group          Address         Size
=======                =====          =====          =======         ====

TEXT32                 CODE           CGROUP         0001:00000000   000f3590
________TEXT           CODE           CGROUP         0001:000f3590   00000000
DATA32                 DATA           DGROUP         0002:00000000   00001cc0
SET1__os2dll           DATA           DGROUP         0002:00001cc0   00000004
SET2__os2dll           DATA           DGROUP         0002:00001cc4   00000000
SET3__os2dll           DATA           DGROUP         0002:00001cc4   00000004
SET1___CTOR_LIST__     DATA           DGROUP         0002:00001cc8   00000004
SET2___CTOR_LIST__     DATA           DGROUP         0002:00001ccc   00000000
SET3___CTOR_LIST__     DATA           DGROUP         0002:00001ccc   00000004
SET1___DTOR_LIST__     DATA           DGROUP         0002:00001cd0   00000004
SET2___DTOR_LIST__     DATA           DGROUP         0002:00001cd4   00000000
SET3___DTOR_LIST__     DATA           DGROUP         0002:00001cd4   00000004
SET1___crtinit1__      DATA           DGROUP         0002:00001cd8   00000004
SET2___crtinit1__      DATA           DGROUP         0002:00001cdc   00000000
SET3___crtinit1__      DATA           DGROUP         0002:00001cdc   00000004
SET1___crtexit1__      DATA           DGROUP         0002:00001ce0   00000004
SET2___crtexit1__      DATA           DGROUP         0002:00001ce4   00000000
SET3___crtexit1__      DATA           DGROUP         0002:00001ce4   00000004
SET1___eh_frame__      DATA           DGROUP         0002:00001ce8   00000004
SET2___eh_frame__      DATA           DGROUP         0002:00001cec   00000008
SET3___eh_frame__      DATA           DGROUP         0002:00001cf4   00000004
SET1___eh_init__       DATA           DGROUP         0002:00001cf8   00000004
SET2___eh_init__       DATA           DGROUP         0002:00001cfc   00000004
SET3___eh_init__       DATA           DGROUP         0002:00001d00   00000004
SET1___eh_term__       DATA           DGROUP         0002:00001d04   00000004
SET2___eh_term__       DATA           DGROUP         0002:00001d08   00000004
SET3___eh_term__       DATA           DGROUP         0002:00001d0c   00000004
SET1___fork_parent1__  DATA           DGROUP         0002:00001d10   00000004
SET2___fork_parent1__  DATA           DGROUP         0002:00001d14   00000000
SET3___fork_parent1__  DATA           DGROUP         0002:00001d14   00000004
SET1___fork_child1__   DATA           DGROUP         0002:00001d18   00000004
SET2___fork_child1__   DATA           DGROUP         0002:00001d1c   00000000
SET3___fork_child1__   DATA           DGROUP         0002:00001d1c   00000004
________DATA           DATA           DGROUP         0002:00001d20   00000000
BSS32                  BSS            DGROUP         0002:00001d20   00000630
c_common               BSS            DGROUP         0002:00002350   00000000
________BSS            BSS            DGROUP         0002:00002350   00000000


                        +----------------+
                        |   Memory Map   |
                        +----------------+

* = unreferenced symbol
+ = symbol only referenced locally

Address        Symbol
=======        ======

Module: U:\usr\lib\dll0hi.obj({standard input})
0001:00000000* __text
0002:00000000* __data
0002:00000000* ___data_start
0002:00001d20* ___bss_start
0002:00001cc0+ __os2dll
0002:00001cc8  ___CTOR_LIST__
0002:00001cd0  ___DTOR_LIST__
0002:00001cd8* ___crtinit1__
0002:00001ce0* ___crtexit1__
0002:00001ce8  ___eh_frame__
0002:00001cf8  ___eh_init__
0002:00001d04  ___eh_term__
0002:00001d10+ ___fork_parent1__
0002:00001d18+ ___fork_child1__
Module: U:/tmp\ldconv__bsddb_obj_ddce4f08029e148440.obj(U:\DEV\python-2.7.2\Modules\_bsddb.c)
0001:000002c9* _DB_length
0001:000019b4  _init_bsddb
0001:00003275+ _init_pybsddb
0001:00003b99* _our_strlcpy
0001:00011288* _DB_subscript
Module: U:\usr\local446\lib\libc_dll.lib(dllinit.obj)
0001:000196b0  _DLL_InitTerm
Module: U:\usr\lib\libend.lib(src/libend/386/endlink386.asm)
0002:00002350  _end
0002:00001d20  _edata
Module: U:\usr\lib\libend.lib(src/libend/386/end.asm)
0001:000f3590* _etext
0001:000f3590* __etext
0000:00000000  WEAK$ZERO
0002:00002350  __end
0002:00001d20  __edata
Module: U:\extras\lib\db-4.5.lib(env_open.obj)
0001:000198f0  ___env_open_pp
0001:00019b30  ___env_open
0001:0001a160* ___env_config
0001:0001a280  ___env_close_pp
0001:0001a3b0  ___env_close
0001:0001a930  ___db_appname
0001:0001af80  _db_version
0001:0001afc0  ___env_remove
0001:0001b0a0  ___env_get_open_flags
Module: U:\extras\lib\db-4.5.lib(db_err.obj)
0001:0001b810  _db_strerror
0001:0001ba10* ___db_unknown_error
0001:0001ba50  ___db_syserr
0001:0001bca0  ___db_errfile
0001:0001bbd0  ___db_errcall
0001:0001bad0  ___db_err
0001:0001bb50  ___db_errx
0001:0001bda0  ___db_msgadd
0001:0001be50  ___db_msg
0001:0001c110  ___db_check_txn
0001:0001c2e0  ___db_txn_deadlock_err
0001:0001c340  ___db_not_txn_env
0001:0001c390  ___db_fchk
0001:0001c3e0  ___db_fcchk
0001:0001c430  ___db_ferr
0001:0001c4c0  ___db_fnl
0001:0001c520  ___db_pgerr
0001:0001c600  ___db_pgfmt
0001:0001c6f0  ___db_panic_msg
0001:0001c760  ___db_panic
0001:0001c7e0  ___db_panic_set
0001:0001c820  ___db_unknown_flag
0001:0001c8a0  ___db_unknown_type
0001:0001c910  ___db_unknown_path
0001:0001c990  ___db_rec_toobig
0001:0001ca20  ___db_rec_repl
0001:0001cab0  ___db_check_lsn
0001:0001cb40  ___db_rdonly
0001:0001cb90  ___db_space_err
0001:0001cbf0  ___db_failed
Module: U:\extras\lib\db-4.5.lib(sequence.obj)
0001:0001cc70  _db_sequence_create
Module: U:\extras\lib\db-4.5.lib(env_method.obj)
0001:0001f2b0  ___env_set_encrypt
0001:0001f8d0  ___db_mi_open
0001:0001f620  ___env_set_flags
0001:0001f990  _db_env_create
0001:0001fac0  ___db_env_destroy
0001:0001fb40  ___env_set_alloc
0001:0001fb80  ___env_get_encrypt_flags
0001:0001fc00  ___env_set_data_dir
0001:0001fd50  ___env_set_intermediate_dir
0001:0001fdb0  ___env_set_errcall
0001:0001fdc0  ___env_get_errfile
0001:0001fdd0  ___env_set_errfile
0001:0001fde0  ___env_get_errpfx
0001:0001fdf0  ___env_set_errpfx
0001:0001fe00  ___env_set_msgcall
0001:0001fe10  ___env_get_msgfile
0001:0001fe20  ___env_set_msgfile
0001:0001fe30  ___env_set_paniccall
0001:0001fe60  ___env_set_shm_key
0001:0001fea0  ___env_set_tmp_dir
0001:0001fef0  ___env_set_verbose
0001:0001ffb0  ___db_mi_env
0001:00020070  ___db_env_config
0002:000019e0  ___db_global_values
Module: U:\extras\lib\db-4.5.lib(db_method.obj)
0001:00020dd0  _db_create
0001:00021680  ___db_get_flags
0001:00021920  ___db_get_lorder
0001:000217f0  ___db_set_flags
0001:00021ad0  ___db_set_pagesize
0001:000219a0* ___db_set_lorder
0001:000215c0  ___dbh_am_chk
Module: U:\usr\local446\lib\gcc\i386-pc-os2-emx\4.4.6\libgcc.lib(emx-ctordtor.obj)
0001:00022350  ___ctordtorTerm
0001:00022382  ___ctordtorInit
Module: U:\extras\lib\db-4.5.lib(os_config.obj)
0001:000223c0* ___os_fs_notzero
0001:000223d0  ___os_support_direct_io
0001:000223e0  ___os_support_db_register
0001:000223f0  ___os_support_replication
Module: U:\extras\lib\db-4.5.lib(env_region.obj)
0001:00022600  ___db_e_attach
0001:00022ed0  ___db_e_detach
0001:000230e0  ___db_e_remove
0001:00023630  ___db_r_attach
0001:00023790  ___db_r_detach
0001:00023a60  ___db_e_golive
Module: U:\extras\lib\db-4.5.lib(mut_region.obj)
0001:00023ac0  ___mutex_open
0001:00024060  ___mutex_dbenv_refresh
Module: U:\extras\lib\db-4.5.lib(env_register.obj)
0001:00024150  ___envreg_register
0001:00024980  ___envreg_unregister
0001:00024a90  ___envreg_xunlock
Module: U:\extras\lib\db-4.5.lib(rep_util.obj)
0001:00024b60  ___rep_bulk_message
0001:000268e0  ___rep_send_throttle
0001:00024df0  ___rep_send_bulk
0001:00024f20  ___rep_send_message
0001:00026b90* ___rep_msg_to_old
0001:00025170  ___rep_new_master
0001:00025d20  ___rep_elect_done
0001:00026840  ___rep_lockout_msg
0001:00025b70  ___rep_noarchive
0001:00025c50  ___rep_send_vote
0001:00025de0  ___rep_grow_sites
0001:00026070  ___env_rep_enter
0001:00026330  ___db_rep_enter
0001:00026580  ___op_rep_enter
0001:00026710  ___rep_lockout_api
0001:00026bb0  ___rep_bulk_alloc
0001:00026c30  ___rep_bulk_free
0001:00026cc0  ___env_db_rep_exit
0001:00026d40  ___op_rep_exit
0001:00026dc0  ___rep_get_gen
0001:00026e50  ___rep_msg_from_old
Module: U:\extras\lib\db-4.5.lib(txn.obj)
0001:00026f20  ___txn_begin_pp
0001:00027120  ___txn_begin
0001:000273a0  ___txn_compensate_begin
0001:000299c0  ___txn_set_timeout
0001:00029990* ___txn_get_name
0001:00029980* ___txn_id
0001:00028490* ___txn_prepare
0001:00028810* ___txn_set_name
0001:00027af0  ___txn_commit
0001:00028090  ___txn_abort
0001:00028340  ___txn_discard_int
0001:00029560  ___txn_force_abort
0001:000296a0  ___txn_preclose
0001:00029760  ___txn_xa_begin
0001:00029800  ___txn_recycle_id
0001:00029910  ___txn_continue
0001:00029a90  ___txn_activekids
0001:00029ae0  ___txn_reset
Module: U:\extras\lib\db-4.5.lib(env_recover.obj)
0001:00029e50  ___db_apprec
0001:0002af80* ___log_backup
0001:0002b290  ___env_openfiles
0001:0002b4c0  ___env_init_rec
Module: U:\extras\lib\db-4.5.lib(mut_alloc.obj)
0001:0002b780  ___mutex_alloc_int
0001:0002b930  ___mutex_free_int
0001:0002b9f0  ___mutex_alloc
0001:0002bb10  ___mutex_free
Module: U:\extras\lib\db-4.5.lib(db_conv.obj)
0001:0002bba0  ___db_pgin
0001:0002bfb0  ___db_pgout
0001:0002c250  ___db_metaswap
0001:0002c4c0  ___db_byteswap
Module: U:\extras\lib\db-4.5.lib(mp_register.obj)
0001:0002cf60  ___memp_register_pp
0001:0002d0a0  ___memp_register
Module: U:\extras\lib\db-4.5.lib(txn_region.obj)
0001:0002d1e0  ___txn_open
0001:0002d540  ___txn_findlastckp
0001:0002d700  ___txn_dbenv_refresh
0001:0002d8a0  ___txn_oldest_reader
0001:0002d9b0  ___txn_remove_buffer
0001:0002dbf0* ___txn_id_set
0001:0002dc80  ___txn_add_buffer
Module: U:\extras\lib\db-4.5.lib(lock_region.obj)
0001:0002ddb0  ___lock_open
0001:0002e560  ___lock_dbenv_refresh
0001:0002e860  ___lock_region_mutex_count
Module: U:\extras\lib\db-4.5.lib(log.obj)
0001:0002e880  ___log_open
0001:0002f1e0  ___log_find
0001:0002f670  ___log_valid
0001:0002fa50  ___log_dbenv_refresh
0001:0002fdd0  ___log_vtruncate
0001:00030210  ___log_zero
0001:00030600  ___log_inmem_lsnoff
0001:00030060  ___log_is_outdated
0001:00030670  ___log_inmem_newfile
0001:00030ac0  ___log_inmem_copyin
0001:00030890  ___log_inmem_chkspace
0001:00030b50  ___log_get_oldversion
0001:00030d30  ___log_get_cached_ckp_lsn
0001:00030dc0  ___log_region_mutex_count
0001:00030de0  ___log_inmem_copyout
0001:00030e70  ___log_set_version
Module: U:\extras\lib\db-4.5.lib(crypto.obj)
0001:00030fc0  ___crypto_region_init
0001:000312d0  ___crypto_algsetup
0001:00031420  ___crypto_decrypt_meta
0001:000315b0  ___crypto_dbenv_close
0001:00031650  ___crypto_region_destroy
0001:000316d0* ___crypto_set_passwd
Module: U:\extras\lib\db-4.5.lib(mp_region.obj)
0001:00031740  ___memp_open
0001:00032110  ___memp_dbenv_refresh
0001:00032510  ___memp_region_mutex_count
Module: U:\extras\lib\db-4.5.lib(rep_region.obj)
0001:00032560  ___rep_open
0001:00032730  ___rep_preclose
0001:000329d0  ___rep_write_egen
0001:00032ae0  ___rep_region_destroy
0001:00032b80  ___rep_dbenv_refresh
0001:00032ba0  ___rep_close
0001:00032c00  ___rep_closefiles
Module: U:\extras\lib\db-4.5.lib(env_failchk.obj)
0001:00032cb0  ___env_failchk_pp
0001:00033240  ___env_set_state
0001:00032ed0  ___env_thread_init
0001:00033540  ___env_thread_id_string
Module: U:\extras\lib\db-4.5.lib(os_alloc.obj)
0001:00033620  ___os_umalloc
0001:00033740  ___os_urealloc
0001:00033840  ___os_ufree
0001:00033880  ___os_strdup
0001:00033950  ___os_calloc
0001:00033a10  ___os_malloc
0001:00033aa0  ___os_realloc
0001:00033ba0  ___os_free
0001:00033bd0  ___ua_memcpy
Module: U:\extras\lib\db-4.5.lib(env_config.obj)
0001:00033c20  ___env_read_db_config
Module: U:\extras\lib\db-4.5.lib(os_tmpdir.obj)
0001:000354a0  ___os_tmpdir
Module: U:\extras\lib\db-4.5.lib(os_oflags.obj)
0001:00035650* ___db_oflags
0001:00035680  ___db_omode
Module: U:\extras\lib\db-4.5.lib(os_root.obj)
0001:00035710  ___os_isroot
Module: U:\extras\lib\db-4.5.lib(os_getenv.obj)
0001:00035770  ___os_getenv
Module: U:\extras\lib\db-4.5.lib(mp_sync.obj)
0001:000357f0  ___memp_walk_files
0001:00035930  ___memp_sync_pp
0001:00035a90  ___memp_sync
0001:00035dd0  ___memp_sync_int
0001:00035c10  ___memp_fsync_pp
0001:00035d50  ___memp_fsync
0001:00036840  ___memp_mf_sync
0001:00036ae0  ___mp_xxx_fh
Module: U:\extras\lib\db-4.5.lib(lock_id.obj)
0001:00036de0  ___lock_id_pp
0001:00036f10  ___lock_id
0001:000373b0  ___lock_getlocker
0001:000370f0  ___lock_id_free_pp
0001:00037250  ___lock_id_free
0001:000378a0* ___lock_freelocker
0001:000375f0  ___lock_addfamilylocker
0001:00037780  ___lock_freefamilylocker
0001:00037980  ___lock_set_thread_id
0001:000379b0* ___lock_id_set
Module: U:\extras\lib\db-4.5.lib(os_abs.obj)
0001:000379f0  ___os_abspath
Module: U:\extras\lib\db-4.5.lib(os_stat.obj)
0001:00037a10  ___os_exists
0001:00037ad0  ___os_ioinfo
Module: U:\extras\lib\db-4.5.lib(os_pid.obj)
0001:00037c10  ___os_id
Module: U:\extras\lib\db-4.5.lib(os_open.obj)
0001:00037c70  ___os_open_extend
0001:00037d90  ___os_open
Module: U:\extras\lib\db-4.5.lib(os_errno.obj)
0001:00037dd0  ___os_get_errno_ret_zero
0001:00037df0  ___os_get_errno
0001:00037e20  ___os_get_syserr
0001:00037e50  ___os_set_errno
0001:00037e90  ___os_strerror
0001:00037ee0  ___os_posix_err
Module: U:\extras\lib\db-4.5.lib(lock.obj)
0001:00037f40  ___lock_vec_pp
0001:000380e0  ___lock_vec
0001:00038ae0  ___lock_get_internal
0001:00038820  ___lock_get_pp
0001:000389a0  ___lock_get
0001:00039730  ___lock_put_pp
0001:00039860  ___lock_put
0001:00039a40  ___lock_downgrade
0001:0003a630  ___lock_promote
0001:0003ab30  ___lock_locker_is_parent
Module: U:\extras\lib\db-4.5.lib(db_pr.obj)
0001:0003ac00* ___db_dumptree
0001:0003dfe0  ___db_dbtype_to_string
0001:0003caa0  ___db_prflags
0001:0003b8e0  ___db_prpage
0001:0003c860  ___db_pr
0001:0003cd20  ___db_dump_pp
0001:0003cea0* ___db_dump
0001:0003d640  ___db_prheader
0001:0003dfb0  ___db_prfooter
0001:0003d1c0  ___db_prdbt
0001:0003e040* ___db_loadme
0001:0003e070* ___db_get_flags_fn
0001:0003e080* ___db_prnpage
0001:0003e1b0  ___db_lockmode_to_string
0001:0003e240  ___db_pr_callback
Module: U:\extras\lib\db-4.5.lib(seq_stat.obj)
0001:0003e9d0  ___seq_stat
0001:0003ecc0  ___seq_stat_print
0001:0003f3d0* ___db_get_seq_flags_fn
Module: U:\extras\lib\db-4.5.lib(db_byteorder.obj)
0001:0003f3f0  ___db_isbigendian
0001:0003f450  ___db_byteorder
Module: U:\extras\lib\db-4.5.lib(db_iface.obj)
0001:0003f500  ___db_associate_pp
0001:00043f00  ___db_txn_auto_resolve
0001:0003fb10  ___db_close_pp
0001:0003fc90  ___db_cursor_pp
0001:0003fe30  ___db_cursor
0001:000400e0  ___db_del_pp
0001:00044020  ___dbt_userfree
0001:00043f70  ___dbt_usercopy
0001:00040410  ___db_fd_pp
0001:000405c0  ___db_get_pp
0001:00040860  ___db_get
0001:00040e10  ___db_join_pp
0001:000410a0  ___db_key_range_pp
0001:00041380  ___db_open_pp
0001:00043ea0  ___db_txn_auto_init
0001:00041c20  ___db_pget_pp
0001:00041e10* ___db_pget
0001:000420d0  ___db_put_pp
0001:000425b0  ___db_compact_pp
0001:00042810  ___db_sync_pp
0001:000429a0  ___db_c_close_pp
0001:00042ad0  ___db_c_count_pp
0001:00042bc0  ___db_c_del_pp
0001:00042d70  ___db_c_dup_pp
0001:00042e40  ___db_c_get_pp
0001:000433c0  ___db_secondary_close_pp
0001:00043530  ___db_c_pget_pp
0001:00043850  ___db_c_put_pp
Module: U:\extras\lib\db-4.5.lib(db_am.obj)
0001:000440e0  ___db_cursor_int
0001:00044620  ___db_put
0001:000447e0  ___db_del
0001:000449e0  ___db_associate
0001:00044ef0  ___db_secondary_close
0001:00045410  ___db_sync
Module: U:\extras\lib\db-4.5.lib(mut_tas.obj)
0001:000454d0  ___db_tas_mutex_lock
0001:00045640  ___db_tas_mutex_init
0001:00045690  ___db_tas_mutex_unlock
0001:000456d0  ___db_tas_mutex_destroy
Module: U:\extras\lib\db-4.5.lib(hmac.obj)
0001:00045760  ___db_check_chksum
0001:00045a10  ___db_chksum
0001:00045c30  ___db_derive_mac
Module: U:\extras\lib\db-4.5.lib(log_method.obj)
0001:00045cd0  ___log_set_lg_max
0001:00045e10  ___log_check_sizes
0001:00045e90  ___log_dbenv_create
0001:00045eb0  ___log_dbenv_destroy
0001:00045ed0  ___log_get_lg_bsize
0001:00045f50  ___log_set_lg_bsize
0001:00045fb0  ___log_get_lg_filemode
0001:000460a0  ___log_set_lg_filemode
0001:00046180  ___log_get_lg_max
0001:00046270  ___log_get_lg_regionmax
0001:00046310  ___log_set_lg_regionmax
0001:00046380  ___log_get_lg_dir
0001:000463a0  ___log_set_lg_dir
0001:000463f0  ___log_get_flags
0001:00046440  ___log_set_flags
Module: U:\extras\lib\db-4.5.lib(lock_method.obj)
0001:00046530  ___lock_set_lk_detect
0001:00046680  ___lock_get_env_timeout
0001:00046800  ___lock_set_env_timeout
0001:00046950  ___lock_dbenv_create
0001:00046970  ___lock_dbenv_destroy
0001:000469c0  ___lock_get_lk_conflicts
0001:00046a70  ___lock_set_lk_conflicts
0001:00046b30  ___lock_get_lk_detect
0001:00046c20  ___lock_get_lk_max_locks
0001:00046ca0  ___lock_set_lk_max_locks
0001:00046d00  ___lock_get_lk_max_lockers
0001:00046d80  ___lock_set_lk_max_lockers
0001:00046de0  ___lock_get_lk_max_objects
0001:00046e60  ___lock_set_lk_max_objects
Module: U:\extras\lib\db-4.5.lib(mp_method.obj)
0001:00046f00  ___memp_set_cachesize
0001:00047030  ___memp_get_mp_max_write
0001:00047120  ___memp_set_mp_max_write
0001:00047210  ___memp_nameop
0001:00047910  ___memp_ftruncate
0001:00047ac0  ___memp_extend_freelist
0001:00047c40  ___memp_dbenv_create
0001:00047c60  ___memp_dbenv_destroy
0001:00047c80  ___memp_get_cachesize
0001:00047d50  ___memp_get_mp_max_openfd
0001:00047e40  ___memp_set_mp_max_openfd
0001:00047f30  ___memp_get_mp_mmapsize
0001:00048000  ___memp_set_mp_mmapsize
0001:000480d0  ___memp_alloc_freelist
0001:00048170  ___memp_free_freelist
0001:00048250  ___memp_get_freelist
Module: U:\extras\lib\db-4.5.lib(rep_method.obj)
0001:000482f0  ___rep_set_config
0001:000486f0  ___rep_start
0001:00048f60  ___rep_client_dbinit
0001:00049920  ___rep_get_limit
0001:00049a30  ___rep_set_limit
0001:00049b30* ___rep_get_request
0001:00049c40  ___rep_set_request
0001:00049e30  ___rep_set_transport
0001:00049f00  ___rep_sync
0001:0004a180  ___rep_dbenv_create
0001:0004a1e0  ___rep_dbenv_destroy
0001:0004a230  ___rep_get_config
0001:0004a350  ___rep_set_nsites
0001:0004a3a0  ___rep_get_nsites
0001:0004a3f0  ___rep_set_priority
0001:0004a440  ___rep_get_priority
0001:0004a4b0  ___rep_set_timeout
0001:0004a550  ___rep_get_timeout
0001:0004a5c0  ___rep_flush
Module: U:\extras\lib\db-4.5.lib(txn_method.obj)
0001:0004a770  ___txn_dbenv_create
0001:0004a790  ___txn_dbenv_destroy
0001:0004a7b0  ___txn_get_tx_max
0001:0004a830  ___txn_set_tx_max
0001:0004a870  ___txn_get_tx_timestamp
0001:0004a8a0  ___txn_set_tx_timestamp
Module: U:\extras\lib\db-4.5.lib(db_cds.obj)
0001:0004a8f0  ___cdsgroup_begin
Module: U:\extras\lib\db-4.5.lib(db_rename.obj)
0001:0004ad90  ___env_dbrename_pp
0001:0004b2c0  ___db_rename_int
0001:0004b060  ___db_rename_pp
0001:0004b210* ___db_rename
Module: U:\extras\lib\db-4.5.lib(db_remove.obj)
0001:0004b6d0  ___env_dbremove_pp
0001:0004bc00  ___db_remove_int
0001:0004b9a0  ___db_remove_pp
0001:0004bb50  ___db_remove
0001:0004be80  ___db_inmem_remove
Module: U:\extras\lib\db-4.5.lib(db_setid.obj)
0001:0004c410  ___env_fileid_reset_pp
Module: U:\extras\lib\db-4.5.lib(lock_stat.obj)
0001:0004ca90  ___lock_stat_pp
0001:0004cde0  ___lock_stat_print_pp
0001:0004cf40  ___lock_stat_print
0001:0004e2e0* ___lock_printlock
Module: U:\extras\lib\db-4.5.lib(lock_deadlock.obj)
0001:0004e650  ___lock_detect_pp
0001:0004e830  ___lock_detect
Module: U:\extras\lib\db-4.5.lib(log_get.obj)
0001:0004fe10  ___log_cursor_pp
0001:0004ff70  ___log_cursor
0001:00050160  ___log_c_close
0001:00050330  ___log_c_version
0001:00050650  ___log_c_get
0001:00051ac0  ___log_rep_split
Module: U:\extras\lib\db-4.5.lib(log_put.obj)
0001:00051c90  ___log_put_pp
0001:00051ee0  ___log_put
0001:00052820  ___log_newfile
0001:00053150  ___log_flush_int
0001:00052e70  ___log_flush_pp
0001:00052fa0  ___log_flush
0001:00053c80  ___log_file_pp
0001:00054050  ___log_name
0001:00054260  ___log_rep_put
0001:000544d0  ___log_current_lsn
Module: U:\extras\lib\db-4.5.lib(log_archive.obj)
0001:000545b0  ___log_archive_pp
0001:00054d00  ___log_get_stable_lsn
0001:00054ec0  ___log_autoremove
Module: U:\extras\lib\db-4.5.lib(log_stat.obj)
0001:00055710  ___log_stat_pp
0001:00055a10  ___log_stat_print_pp
0001:00055b70  ___log_stat_print
Module: U:\extras\lib\db-4.5.lib(log_debug.obj)
0001:00056970  ___log_printf_capi
0001:000569b0* ___log_printf_pp
0001:00056af0* ___log_printf
Module: U:\extras\lib\db-4.5.lib(mp_fmethod.obj)
0001:00056c90  ___memp_fcreate_pp
0001:00056dc0  ___memp_fcreate
0001:00057130  ___memp_get_ftype
0001:00056f00  ___memp_set_flags
0001:00057160  ___memp_set_ftype
0001:000571c0  ___memp_set_lsn_offset
0001:00057220  ___memp_set_pgcookie
0001:00057010  ___memp_get_fileid
0001:000570f0  ___memp_get_flags
0001:00056fb0  ___memp_set_clear_len
0001:00057080  ___memp_set_fileid
0001:000572f0  ___memp_last_pgno
0001:00057370  ___memp_fn
0001:000573b0  ___memp_fns
Module: U:\extras\lib\db-4.5.lib(db_setlsn.obj)
0001:00057810  ___env_lsn_reset_pp
Module: U:\extras\lib\db-4.5.lib(mp_stat.obj)
0001:00057b20  ___memp_stat_pp
0001:0005a700  ___memp_stat_hash
0001:000582a0  ___memp_stat_print_pp
0001:00058400  ___memp_stat_print
Module: U:\extras\lib\db-4.5.lib(mut_method.obj)
0001:0005a7c0  ___mutex_alloc_pp
0001:0005a8b0  ___mutex_free_pp
0001:0005a950  ___mutex_lock_pp
0001:0005a9a0  ___mutex_unlock_pp
0001:0005a9f0  ___mutex_get_align
0001:0005aa90  ___mutex_set_align
0001:0005ab00  ___mutex_get_increment
0001:0005ab30  ___mutex_set_increment
0001:0005ab80  ___mutex_get_max
0001:0005abc0  ___mutex_set_max
0001:0005ac10  ___mutex_get_tas_spins
0001:0005ac40  ___mutex_set_tas_spins
Module: U:\extras\lib\db-4.5.lib(mp_trickle.obj)
0001:0005ac90  ___memp_trickle_pp
Module: U:\extras\lib\db-4.5.lib(mut_stat.obj)
0001:0005af80  ___mutex_stat
0001:0005b750  ___mutex_set_wait_info
0001:0005b780  ___mutex_clear
0001:0005b180  ___mutex_print_debug_single
0001:0005b270  ___mutex_print_debug_stats
0001:0005b7f0  ___mutex_stat_print
Module: U:\extras\lib\db-4.5.lib(rep_elect.obj)
0001:0005c1e0  ___rep_elect
0001:0005d3a0* ___rep_elect_master
0001:0005c9c0  ___rep_vote1
0001:0005ce30  ___rep_vote2
Module: U:\extras\lib\db-4.5.lib(rep_stat.obj)
0001:0005d520  ___rep_stat_pp
0001:0005d8c0  ___rep_stat_print_pp
0001:0005d9b0  ___rep_stat_print
Module: U:\extras\lib\db-4.5.lib(rep_record.obj)
0001:0005f9e0  ___rep_process_message
0001:00060df0  ___rep_apply
0001:00062650  ___rep_check_doreq
0001:00061710  ___rep_process_txn
Module: U:\extras\lib\db-4.5.lib(env_stat.obj)
0001:00062860  ___env_stat_print_pp
0001:00064430  ___db_dlbytes
0001:000641c0  ___db_print_fileid
0001:00064300  ___db_dl_pct
0001:000647e0  ___db_print_fh
0001:00064960  ___db_dl
0001:00064ad0  ___db_print_reginfo
Module: U:\extras\lib\db-4.5.lib(txn_chkpt.obj)
0001:00064c90  ___txn_checkpoint_pp
0001:00064e70  ___txn_checkpoint
0001:00065210  ___txn_getactive
0001:000652f0  ___txn_updateckp
0001:000653a0  ___txn_getckp
Module: U:\extras\lib\db-4.5.lib(txn_recover.obj)
0001:000654a0  ___txn_recover_pp
0001:00065650  ___txn_recover
0001:00065690  ___txn_get_prepared
0001:00065af0  ___txn_openfiles
0001:00065d90  ___txn_map_gid
Module: U:\extras\lib\db-4.5.lib(txn_stat.obj)
0001:00065ec0  ___txn_stat_pp
0001:00066380  ___txn_stat_print_pp
0001:000664e0  ___txn_stat_print
Module: U:\extras\lib\db-4.5.lib(mp_fopen.obj)
0001:00067580  ___memp_fopen_pp
0001:00067830  ___memp_fopen
0001:00068da0  ___memp_mf_discard
0001:00068870  ___memp_fclose_pp
0001:000689b0  ___memp_fclose
0001:00069090  ___memp_inmemlist
Module: U:\extras\lib\db-4.5.lib(db_open.obj)
0001:00069360  ___db_open
0001:000697f0  ___db_new_file
0001:00069910  ___db_init_subdb
0001:00069d30  ___db_meta_setup
0001:00069a50  ___db_chk_meta
0001:0006a010  ___db_get_open_flags
Module: U:\extras\lib\db-4.5.lib(db_stati.obj)
0001:0006a070  ___db_stat_pp
0001:0006a1f0* ___db_stat
0001:0006a350  ___db_stat_print_pp
0001:0006a4e0  ___db_stat_print
Module: U:\extras\lib\db-4.5.lib(db_upg.obj)
0001:0006b830* ___db_upgrade
0001:0006bfd0  ___db_lastpgno
0001:0006c190  ___db_upgrade_pp
Module: U:\extras\lib\db-4.5.lib(db_truncate.obj)
0001:0006c2d0  ___db_truncate_pp
0001:0006c560  ___db_truncate
Module: U:\extras\lib\db-4.5.lib(db_vrfy.obj)
0001:0006da30  ___db_vrfy_common
0001:0006f190  ___db_salvage
0001:0006dd60  ___db_vrfy_datapage
0001:0006e180  ___db_vrfy_meta
0001:0006f8d0  ___db_vrfy_inpitem
0001:0006fc40  ___db_vrfy_duptype
0001:0006fdb0  ___db_salvage_duptree
0001:000709d0  ___db_verify_pp
0001:00070ae0* ___db_verify_internal
0001:00070c00  ___db_vrfy_struct_feedback
Module: U:\extras\lib\db-4.5.lib(bt_method.obj)
0001:00071280  ___bam_map_flags
0001:00071300  ___bam_set_flags
0001:00071430  ___bam_db_create
0001:000715b0  ___bam_set_bt_compare
0001:00071630  ___bam_get_bt_minkey
0001:00071770  ___ram_get_re_len
0001:000717c0  ___ram_get_re_pad
0001:00071530  ___bam_db_close
0001:00071670  ___ram_map_flags
0001:000716b0  ___ram_set_flags
Module: U:\extras\lib\db-4.5.lib(hash_method.obj)
0001:00071c00  ___ham_db_create
0001:00071cd0  ___ham_get_h_ffactor
0001:00071cf0  ___ham_get_h_nelem
0001:00071c90  ___ham_db_close
Module: U:\extras\lib\db-4.5.lib(qam_method.obj)
0001:00071eb0  ___qam_db_close
0001:00071ff0  ___db_prqueue
0001:00072230  ___qam_db_create
0001:000722a0  ___qam_get_extentsize
0001:000722c0  ___queue_pageinfo
0001:000723f0  ___qam_remove
0001:00072430  ___qam_rename
0001:00072470  ___qam_map_flags
0001:00072490  ___qam_set_flags
Module: U:\extras\lib\db-4.5.lib(xa_db.obj)
0001:00072770  ___db_xa_create
Module: U:\tmp\ldconv_libgcc_so_d_a_ddce4f08029e1635d8.lib(emx-eh.obj)
0001:00072dc5  ___ehInit
0001:00072d90* ___ehTerm
Module: U:\extras\lib\db-4.5.lib(os_region.obj)
0001:00072e00  ___os_r_attach
0001:00072ee0  ___os_r_detach
Module: U:\extras\lib\db-4.5.lib(os_sleep.obj)
0001:00072f90  ___os_sleep
Module: U:\extras\lib\db-4.5.lib(os_handle.obj)
0001:00073060  ___os_openhandle
0001:00073270  ___os_closehandle
Module: U:\extras\lib\db-4.5.lib(db_salloc.obj)
0001:00073350  ___db_shalloc
0001:000734b0  ___db_shalloc_free
0001:00073720  ___db_shalloc_init
0001:00073760  ___db_shalloc_size
0001:00073790  ___db_shalloc_sizeof
Module: U:\extras\lib\db-4.5.lib(os_uid.obj)
0001:000737b0  ___os_unique_id
Module: U:\extras\lib\db-4.5.lib(os_rw.obj)
0001:00073840  ___os_io
0001:00073b60  ___os_write
0001:00073a30  ___os_read
0001:00073b80* ___os_physwrite
Module: U:\extras\lib\db-4.5.lib(os_rpath.obj)
0001:00073d40  ___db_rpath
Module: U:\extras\lib\db-4.5.lib(os_dir.obj)
0001:00073d80  ___os_dirlist
0001:00073fa0  ___os_dirfree
Module: U:\extras\lib\db-4.5.lib(os_unlink.obj)
0001:00074010  ___os_unlink
0001:000740b0* ___os_region_unlink
Module: U:\extras\lib\db-4.5.lib(env_file.obj)
0001:000740f0* ___db_file_write
0001:00074240  ___db_file_extend
0001:000742f0  ___db_file_multi_write
Module: U:\extras\lib\db-4.5.lib(os_spin.obj)
0001:00074420  ___os_spin
Module: U:\extras\lib\db-4.5.lib(os_flock.obj)
0001:00074460  ___os_fdlock
Module: U:\extras\lib\db-4.5.lib(os_seek.obj)
0001:00074550  ___os_seek
Module: U:\extras\lib\db-4.5.lib(rep_backup.obj)
0001:00074660  ___rep_update_req
0001:00075460  ___rep_page_req
0001:00075e90  ___rep_update_setup
0001:00076480  ___rep_bulk_page
0001:00076540  ___rep_page
0001:000767d0  ___rep_page_fail
0001:00076b20  ___rep_init_cleanup
0001:00076fc0  ___rep_pggap_req
0001:00077200* ___rep_finfo_alloc
Module: U:\extras\lib\db-4.5.lib(rep_verify.obj)
0001:00077850  ___rep_verify
0001:00078490  ___rep_log_backup
0001:00077ff0  ___rep_verify_match
0001:00077c00  ___rep_verify_fail
0001:00077ed0  ___rep_verify_req
Module: U:\extras\lib\db-4.5.lib(os_clock.obj)
0001:000786d0  ___os_clock
Module: U:\extras\lib\db-4.5.lib(db_clock.obj)
0001:00078790  ___db_difftime
Module: U:\extras\lib\db-4.5.lib(lock_timer.obj)
0001:000787d0  ___lock_set_timeout_internal
0001:00078a20  ___lock_expires
0001:00078900  ___lock_inherit_timeout
0001:00078a90  ___lock_set_timeout
0001:00078b20  ___lock_expired
Module: U:\extras\lib\db-4.5.lib(txn_auto.obj)
0001:00078b90  ___txn_regop_42_read
0001:00078c40  ___txn_regop_log
0001:00078f40  ___txn_regop_read
0001:00078ff0  ___txn_ckp_log
0001:00079300  ___txn_ckp_read
0001:000793b0  ___txn_child_log
0001:00079680  ___txn_xa_regop_log
0001:00079a00  ___txn_xa_regop_read
0001:00079af0  ___txn_recycle_log
0001:00079d90  ___txn_ckp_42_read
0001:00079e30  ___txn_child_read
0001:00079ec0  ___txn_recycle_read
0001:00079f50  ___txn_init_recover
Module: U:\extras\lib\db-4.5.lib(db_idspace.obj)
0001:0007a050  ___db_idspace
Module: U:\extras\lib\db-4.5.lib(db_dispatch.obj)
0001:0007a180  ___db_dispatch
0001:0007a690  ___db_txnlist_add
0001:0007a840  ___db_txnlist_find
0001:0007a890  ___db_txnlist_update
0001:0007a500  ___db_txnlist_init
0001:0007a780  ___db_txnlist_end
0001:0007aba0  ___db_txnlist_lsnadd
0001:0007acc0* ___db_txnlist_lsninit
0001:0007ac70  ___db_txnlist_lsnget
0001:0007b1b0  ___db_add_recovery
0001:0007b230  ___db_txnlist_remove
0001:0007b280  ___db_txnlist_ckp
0001:0007b2d0  ___db_txnlist_gen
0001:0007b390  ___db_add_limbo
0001:0007b470* ___db_do_the_limbo
Module: U:\extras\lib\db-4.5.lib(txn_util.obj)
0001:0007bf20  ___txn_remevent
0001:0007c040  ___txn_doevents
0001:0007c330  ___txn_closeevent
0001:0007c3a0  ___txn_remrem
0001:0007c440  ___txn_lockevent
0001:0007c4f0  ___txn_remlock
Module: U:\extras\lib\db-4.5.lib(dbreg_util.obj)
0001:0007c570  ___dbreg_add_dbentry
0001:0007c660  ___dbreg_log_files
0001:0007c810  ___dbreg_close_files
0001:0007c970  ___dbreg_invalidate_files
0001:0007ca50  ___dbreg_id_to_db_int
0001:0007cc10  ___dbreg_id_to_fname
0001:0007cdd0  ___dbreg_do_open
0001:0007ccd0  ___dbreg_fid_to_fname
0001:0007d1a0  ___dbreg_lazy_id
0001:0007d320  ___dbreg_rem_dbentry
0001:0007d3a0  ___dbreg_id_to_db
0001:0007d3e0  ___dbreg_get_name
Module: U:\extras\lib\db-4.5.lib(ctime.obj)
0001:0007d450  ___db_ctime
Module: U:\extras\lib\db-4.5.lib(btree_auto.obj)
0001:0007d480  ___bam_split_log
0001:0007d990  ___bam_split_read
0001:0007da80  ___bam_rsplit_log
0001:0007deb0  ___bam_rsplit_read
0001:0007dfa0  ___bam_adj_log
0001:0007e330  ___bam_adj_read
0001:0007e3e0  ___bam_cadjust_log
0001:0007e770  ___bam_cadjust_read
0001:0007e820  ___bam_cdel_log
0001:0007eba0  ___bam_cdel_read
0001:0007ec40  ___bam_repl_log
0001:0007f080  ___bam_repl_read
0001:0007f170  ___bam_root_log
0001:0007f4f0  ___bam_root_read
0001:0007f590  ___bam_curadj_log
0001:0007f8a0  ___bam_curadj_read
0001:0007f950  ___bam_rcuradj_log
0001:0007fc50  ___bam_rcuradj_read
0001:0007fcf0  ___bam_relink_43_read
0001:0007fdb0  ___bam_relink_log
0001:000801e0  ___bam_relink_read
0001:00080290  ___bam_merge_log
0001:000807a0  ___bam_merge_read
0001:000808b0  ___bam_pgno_log
0001:00080c40  ___bam_pgno_read
0001:00080cf0  ___bam_init_recover
Module: U:\extras\lib\db-4.5.lib(crdel_auto.obj)
0001:00080f10  ___crdel_metasub_log
0001:000812e0  ___crdel_metasub_read
0001:00081390  ___crdel_inmem_create_log
0001:000816e0  ___crdel_inmem_create_read
0001:000817b0  ___crdel_inmem_rename_log
0001:00081b40  ___crdel_inmem_rename_read
0001:00081c30  ___crdel_inmem_remove_log
0001:00081f60  ___crdel_inmem_remove_read
0001:00082020  ___crdel_init_recover
Module: U:\extras\lib\db-4.5.lib(db_auto.obj)
0001:000820f0  ___db_addrem_log
0001:00082520  ___db_addrem_read
0001:00082610  ___db_big_log
0001:00082b10  ___db_big_read
0001:00082c00  ___db_ovref_log
0001:00082f80  ___db_ovref_read
0001:00083020  ___db_relink_42_read
0001:000830e0  ___db_debug_log
0001:00083470  ___db_debug_read
0001:00083570* ___db_noop_log
0001:000838f0  ___db_pg_alloc_42_read
0001:000839a0  ___db_pg_alloc_log
0001:00083dd0  ___db_pg_alloc_read
0001:00083e80  ___db_pg_free_42_read
0001:00083f40  ___db_pg_free_log
0001:00084330  ___db_pg_free_read
0001:00084400  ___db_cksum_log
0001:00084690  ___db_pg_freedata_42_read
0001:00084770  ___db_pg_freedata_log
0001:00084ba0  ___db_pg_freedata_read
0001:00084c90  ___db_pg_prepare_log
0001:00084f70  ___db_pg_new_log
0001:00085360* ___db_pg_new_read
0001:00085420  ___db_pg_init_log
0001:000857a0  ___db_pg_init_read
0001:00085870  ___db_pg_sort_log
0001:00085ce0  ___db_pg_sort_read
0001:00085db0  ___db_init_recover
0001:00086000  ___db_noop_read
0001:00086090  ___db_cksum_read
0001:00086110* ___db_pg_prepare_read
Module: U:\extras\lib\db-4.5.lib(dbreg_auto.obj)
0001:000861a0  ___dbreg_register_log
0001:00086500  ___dbreg_register_read
0001:000865e0  ___dbreg_init_recover
Module: U:\extras\lib\db-4.5.lib(fileops_auto.obj)
0001:00086630  ___fop_create_log
0001:00086920  ___fop_create_read
0001:000869d0  ___fop_remove_log
0001:00086d10  ___fop_remove_read
0001:00086dd0  ___fop_write_log
0001:00087130  ___fop_write_read
0001:00087210  ___fop_rename_log
0001:000875b0  ___fop_rename_read
0001:000876a0  ___fop_file_remove_log
0001:00087a40  ___fop_file_remove_read
0001:00087b40  ___fop_init_recover
Module: U:\extras\lib\db-4.5.lib(hash_auto.obj)
0001:00087c40  ___ham_insdel_log
0001:00088070  ___ham_insdel_read
0001:00088150  ___ham_newpage_log
0001:00088600  ___ham_newpage_read
0001:000886c0  ___ham_splitdata_log
0001:00088aa0  ___ham_splitdata_read
0001:00088b60  ___ham_replace_log
0001:00088fa0  ___ham_replace_read
0001:00089090  ___ham_copypage_log
0001:00089580  ___ham_copypage_read
0001:00089660  ___ham_metagroup_42_read
0001:00089730  ___ham_metagroup_log
0001:00089bf0  ___ham_metagroup_read
0001:00089cc0  ___ham_groupalloc_42_read
0001:00089d60  ___ham_groupalloc_log
0001:0008a0f0  ___ham_groupalloc_read
0001:0008a1a0  ___ham_curadj_log
0001:0008a4b0  ___ham_curadj_read
0001:0008a560  ___ham_chgpg_log
0001:0008a860  ___ham_chgpg_read
0001:0008a900  ___ham_init_recover
Module: U:\extras\lib\db-4.5.lib(qam_auto.obj)
0001:0008aab0  ___qam_incfirst_log
0001:0008ada0  ___qam_mvptr_log
0001:0008b140  ___qam_mvptr_read
0001:0008b1f0  ___qam_del_log
0001:0008b580  ___qam_del_read
0001:0008b620  ___qam_add_log
0001:0008ba50  ___qam_add_read
0001:0008bb40  ___qam_delext_log
0001:0008bf10  ___qam_delext_read
0001:0008bfd0  ___qam_incfirst_read
0001:0008c060  ___qam_init_recover
Module: U:\extras\lib\db-4.5.lib(db_rec.obj)
0001:0008c160  ___db_addrem_recover
0001:0008c590  ___db_big_recover
0001:0008cda0  ___db_ovref_recover
0001:0008d080  ___db_debug_recover
0001:0008d0e0  ___db_noop_recover
0001:0008d3b0  ___db_pg_alloc_recover
0001:0008db60  ___db_pg_free_recover
0001:0008dc50  ___db_pg_new_recover
0001:0008dc60  ___db_pg_freedata_recover
0001:0008dd90  ___db_cksum_recover
0001:0008de10  ___db_pg_prepare_recover
0001:0008de20  ___db_pg_init_recover
0001:0008e1d0  ___db_pg_sort_recover
0001:0008e810  ___db_pg_alloc_42_recover
0001:0008ef50  ___db_pg_free_42_recover
0001:0008f040  ___db_pg_freedata_42_recover
0001:0008f130  ___db_relink_42_recover
Module: U:\extras\lib\db-4.5.lib(hash_rec.obj)
0001:00090700  ___ham_insdel_recover
0001:00090bc0  ___ham_newpage_recover
0001:00091400  ___ham_replace_recover
0001:000917e0  ___ham_splitdata_recover
0001:00091bb0  ___ham_copypage_recover
0001:000922e0  ___ham_metagroup_recover
0001:00092c60  ___ham_groupalloc_recover
0001:00093270  ___ham_curadj_recover
0001:000933e0  ___ham_chgpg_recover
0001:00093880  ___ham_metagroup_42_recover
0001:000940d0  ___ham_groupalloc_42_recover
Module: U:\extras\lib\db-4.5.lib(txn_rec.obj)
0001:000946c0  ___txn_regop_recover
0001:000948c0  ___txn_xa_regop_recover
0001:00094db0  ___txn_restore_txn
0001:00094ab0  ___txn_child_recover
0001:00094fd0  ___txn_regop_42_recover
0001:000951b0  ___txn_ckp_recover
0001:00095260  ___txn_recycle_recover
0001:00095300  ___txn_ckp_42_recover
Module: U:\extras\lib\db-4.5.lib(bt_rec.obj)
0001:000953c0  ___bam_split_recover
0001:00096230  ___bam_rsplit_recover
0001:00096850  ___bam_adj_recover
0001:00096c00  ___bam_cadjust_recover
0001:00097070  ___bam_cdel_recover
0001:00097400  ___bam_repl_recover
0001:00097980  ___bam_root_recover
0001:00097c70  ___bam_curadj_recover
0001:00097e40  ___bam_rcuradj_recover
0001:00098050  ___bam_relink_recover
0001:00098510  ___bam_merge_recover
0001:00098e30  ___bam_pgno_recover
0001:00099240  ___bam_relink_43_recover
Module: U:\extras\lib\db-4.5.lib(hash_conv.obj)
0001:00099860  ___ham_mswap
0001:00099a30  ___ham_pgin
0001:00099ae0  ___ham_pgout
Module: U:\extras\lib\db-4.5.lib(qam_conv.obj)
0001:00099b60  ___qam_mswap
0001:00099cf0  ___qam_pgin_out
Module: U:\extras\lib\db-4.5.lib(bt_conv.obj)
0001:00099d80  ___bam_mswap
0001:00099ea0  ___bam_pgin
0001:00099f20  ___bam_pgout
Module: U:\extras\lib\db-4.5.lib(db_shash.obj)
0001:0009a0e0  ___db_tablesize
0001:0009a120  ___db_hashinit
Module: U:\usr\local446\lib\gcc\i386-pc-os2-emx\4.4.6\libgcc.lib(_alloca.obj)
0001:0009a160  __alloca
Module: U:\extras\lib\db-4.5.lib(aes_method.obj)
0001:0009a190  ___aes_setup
0001:0009a200* ___aes_adj_size
0001:0009a220* ___aes_close
0001:0009a240* ___aes_decrypt
0001:0009a2e0* ___aes_encrypt
0001:0009a400* ___aes_init
Module: U:\extras\lib\db-4.5.lib(mp_bh.obj)
0001:0009a740  ___memp_bhwrite
0001:0009aaf0  ___memp_pgread
0001:0009b000  ___memp_pg
0001:0009b1b0  ___memp_bhfree
Module: U:\extras\lib\db-4.5.lib(mp_alloc.obj)
0001:0009b5e0  ___memp_alloc
0001:0009c690  ___memp_free
Module: U:\extras\lib\db-4.5.lib(db.obj)
0001:0009c6d0  ___db_master_update
0001:0009ccc0  ___db_dbenv_setup
0001:0009d090  ___db_dbenv_mpool
0001:0009d3c0  ___db_close
0001:0009d4e0  ___db_refresh
0001:0009dce0  ___db_backup_name
0001:0009dfd0  ___db_master_open
0001:0009e0e0  ___db_log_page
Module: U:\extras\lib\db-4.5.lib(os_fsync.obj)
0001:0009e1a0  ___os_fsync
Module: U:\extras\lib\db-4.5.lib(txn_failchk.obj)
0001:0009e2a0  ___txn_failchk
Module: U:\extras\lib\db-4.5.lib(mut_failchk.obj)
0001:0009e640  ___mut_failchk
Module: U:\extras\lib\db-4.5.lib(lock_failchk.obj)
0001:0009e830  ___lock_failchk
Module: U:\extras\lib\db-4.5.lib(db_getlong.obj)
0001:0009ebe0  ___db_getlong
0001:0009ee90  ___db_getulong
Module: U:\extras\lib\db-4.5.lib(lock_util.obj)
0001:0009f060  ___lock_ohash
0001:0009f0c0  ___lock_lhash
0001:0009f150  ___lock_nomem
Module: U:\extras\lib\db-4.5.lib(mkpath.obj)
0001:0009f180  ___db_mkpath
Module: U:\extras\lib\db-4.5.lib(lock_list.obj)
0001:0009f260  ___lock_fix_list
0001:0009f5b0  ___lock_get_list
0001:0009f7b0* ___lock_list_print
Module: U:\extras\lib\db-4.5.lib(mp_fget.obj)
0001:0009f990  ___memp_fget_pp
0001:0009fca0  ___memp_fget
Module: U:\extras\lib\db-4.5.lib(mp_fput.obj)
0001:000a1c10  ___memp_fput_pp
0001:000a1d60  ___memp_fput
Module: U:\extras\lib\db-4.5.lib(db_cam.obj)
0001:000a2310  ___db_c_close
0001:000a2580  ___db_c_destroy
0001:000a26d0  ___db_c_del
0001:000a5490  ___db_c_del_primary
0001:000a28a0  ___db_c_idup
0001:000a2a70  ___db_c_get
0001:000a3510  ___db_c_put
0001:000a5880  ___db_s_first
0001:000a5900  ___db_s_next
0001:000a59d0  ___db_s_done
0001:000a4a20  ___db_c_pget
0001:000a5c40  ___db_partsize
0001:000a5c90  ___db_c_count
0001:000a5d30  ___db_c_dup
0001:000a5df0  ___db_c_newopd
0001:000a5ed0  ___db_duperr
0001:000a5f10  ___db_c_secondary_get_pp
Module: U:\extras\lib\db-4.5.lib(db_vrfyutil.obj)
0001:000a5f50  ___db_vrfy_dbinfo_create
0001:000a64c0  ___db_vrfy_pgset
0001:000a61c0  ___db_vrfy_dbinfo_destroy
0001:000a63e0  ___db_vrfy_putpageinfo
0001:000a62f0  ___db_vrfy_getpageinfo
0001:000a65a0  ___db_vrfy_childput
0001:000a6750  ___db_vrfy_ccset
0001:000a67c0  ___db_vrfy_ccnext
0001:000a6820  ___db_vrfy_ccclose
0001:000a6880  ___db_vrfy_pgset_get
0001:000a6910  ___db_vrfy_pgset_inc
0001:000a69c0  ___db_vrfy_pgset_next
0001:000a6a40  ___db_vrfy_childcursor
0001:000a6a80  ___db_salvage_init
0001:000a6b40  ___db_salvage_destroy
0001:000a6b70  ___db_salvage_getnext
0001:000a6c50  ___db_salvage_isdone
0001:000a6cf0  ___db_salvage_markdone
0001:000a6e50  ___db_salvage_markneeded
0001:000a6ee0  ___db_vrfy_prdbt
Module: U:\extras\lib\db-4.5.lib(db_join.obj)
0001:000a6fa0  ___db_join
0001:000a7c30  ___db_join_close
0001:000a80c0  ___db_secondary_corrupt
Module: U:\extras\lib\db-4.5.lib(bt_stat.obj)
0001:000a81c0  ___bam_stat
0001:000a9180  ___bam_stat_callback
0001:000a9650  ___bam_traverse
0001:000a8c30  ___bam_stat_print
0001:000a94e0  ___bam_key_range
0001:000a9ce0  ___bam_print_cursor
Module: U:\extras\lib\db-4.5.lib(bt_compact.obj)
0001:000a9dc0  ___bam_compact
Module: U:\extras\lib\db-4.5.lib(bt_cursor.obj)
0001:000aee00  ___bam_c_init
0001:000aef40  ___bam_c_refresh
0001:000af730  ___bam_c_count
0001:000b0f10  ___bam_bulk_overflow
0001:000b0f80  ___bam_bulk_duplicates
0001:000b3620  ___bam_opd_exists
0001:000b3690  ___bam_c_dup
0001:000b36d0  ___bam_c_rget
Module: U:\extras\lib\db-4.5.lib(hash.obj)
0001:000b3950  ___ham_c_init
0001:000b3c50  ___ham_c_count
0001:000b67a0  ___ham_c_update
0001:000b6730  ___ham_init_dbt
0001:000b6de0  ___ham_get_clist
0001:000b7090  ___ham_quick_delete
0001:000b7190  ___ham_c_dup
0001:000b71f0  ___ham_call_hash
Module: U:\extras\lib\db-4.5.lib(qam.obj)
0001:000b7350  ___qam_position
0001:000b75b0  ___qam_pitem
0001:000b79a0  ___qam_append
0001:000b8460  ___qam_truncate
0001:000b86a0  ___qam_c_dup
0001:000b86c0  ___qam_c_init
0001:000b87c0  ___qam_delete
Module: U:\extras\lib\db-4.5.lib(bt_recno.obj)
0001:000bac80  ___ram_c_del
0001:000bbb30  ___ram_ca
0001:000bb030  ___ram_c_get
0001:000bc0d0  ___ram_getno
0001:000bb540  ___ram_c_put
0001:000bc280  ___ram_writeback
0001:000bc9f0  ___ram_open
0001:000bcb70  ___ram_append
Module: U:\extras\lib\db-4.5.lib(bt_compare.obj)
0001:000bcc30  ___bam_cmp
0001:000bcdd0  ___bam_defcmp
0001:000bce40  ___bam_defpfx
Module: U:\extras\lib\db-4.5.lib(qam_files.obj)
0001:000bceb0  ___qam_fprobe
0001:000bdfb0* ___qam_exid
0001:000bd8d0  ___qam_fclose
0001:000bd990  ___qam_fremove
0001:000bdb10* ___qam_gen_filelist
0001:000bdce0  ___qam_extent_names
0001:000be020  ___qam_nameop
0001:000be660  ___qam_sync
Module: U:\extras\lib\db-4.5.lib(sha1.obj)
0001:000be6a0* ___db_SHA1Transform
0001:000c0100  ___db_SHA1Init
0001:000c0140  ___db_SHA1Update
0001:000c0210  ___db_SHA1Final
Module: U:\extras\lib\db-4.5.lib(hash_func.obj)
0001:000c04f0* ___ham_func3
0001:000c05c0  ___ham_func4
0001:000c06a0* ___ham_func2
0001:000c06f0  ___ham_func5
0001:000c0730* ___ham_test
Module: U:\extras\lib\db-4.5.lib(os_rename.obj)
0001:000c0750  ___os_rename
Module: U:\extras\lib\db-4.5.lib(os_truncate.obj)
0001:000c0810  ___os_truncate
Module: U:\extras\lib\db-4.5.lib(fop_util.obj)
0001:000c08e0  ___fop_lock_handle
0001:000c0b20  ___fop_file_setup
0001:000c2430  ___fop_read_meta
0001:000c1c90  ___fop_subdb_setup
0001:000c1fe0  ___fop_remove_setup
0001:000c2500  ___fop_dummy
0001:000c27a0  ___fop_dbrename
Module: U:\extras\lib\db-4.5.lib(fop_basic.obj)
0001:000c3a10  ___fop_create
0001:000c3ba0  ___fop_remove
0001:000c3d30  ___fop_write
0001:000c3f20  ___fop_rename
Module: U:\extras\lib\db-4.5.lib(bt_reclaim.obj)
0001:000c40f0  ___bam_reclaim
0001:000c41e0  ___bam_truncate
Module: U:\extras\lib\db-4.5.lib(hash_reclaim.obj)
0001:000c4240  ___ham_reclaim
0001:000c4340  ___ham_truncate
Module: U:\extras\lib\db-4.5.lib(os_fid.obj)
0001:000c43e0  ___os_fileid
Module: U:\extras\lib\db-4.5.lib(db_ret.obj)
0001:000c4550  ___db_ret
0001:000c4720  ___db_retcopy
Module: U:\extras\lib\db-4.5.lib(mp_fset.obj)
0001:000c48e0  ___memp_fset_pp
0001:000c4a80* ___memp_fset
0001:000c4c50  ___memp_dirty
Module: U:\extras\lib\db-4.5.lib(rep_log.obj)
0001:000c4f00  ___rep_allreq
0001:000c5380  ___rep_log
0001:000c5b20  ___rep_loggap_req
0001:000c5d60  ___rep_logready
0001:000c5650  ___rep_logreq
0001:000c6020  ___rep_bulk_log
Module: U:\extras\lib\db-4.5.lib(dbreg_stat.obj)
0001:000c60a0  ___dbreg_stat_print
0001:000c6160  ___dbreg_print_fname
Module: U:\extras\lib\db-4.5.lib(os_map.obj)
0001:000c6640  ___os_r_sysattach
0001:000c6850  ___os_r_sysdetach
0001:000c6930  ___os_mapfile
0001:000c69a0  ___os_unmapfile
Module: U:\extras\lib\db-4.5.lib(bt_open.obj)
0001:000c6cc0  ___bam_metachk
0001:000c7000  ___bam_read_root
0001:000c7190  ___bam_new_file
0001:000c7620  ___bam_new_subdb
0001:000c79d0  ___bam_open
Module: U:\extras\lib\db-4.5.lib(hash_open.obj)
0001:000c7cf0  ___ham_open
0001:000c8030  ___ham_metachk
0001:000c8240  ___ham_new_file
0001:000c8680  ___ham_new_subdb
Module: U:\extras\lib\db-4.5.lib(qam_open.obj)
0001:000c8da0  ___qam_open
0001:000c9020  ___qam_set_ext_data
0001:000c9140  ___qam_metachk
0001:000c92a0  ___qam_new_file
Module: U:\extras\lib\db-4.5.lib(dbreg.obj)
0001:000c96c0  ___dbreg_setup
0001:000c9890  ___dbreg_new_id
0001:000c9960  ___dbreg_get_id
0001:000ca350  ___dbreg_log_id
0001:000c9d00  ___dbreg_revoke_id
0001:000c9ae0  ___dbreg_assign_id
0001:000c9e70  ___dbreg_close_id
0001:000c9f60  ___dbreg_log_close
0001:000ca520  ___dbreg_teardown
Module: U:\extras\lib\db-4.5.lib(log_compare.obj)
0001:000ca600  _log_compare
0001:000ca780  ___log_check_page_lsn
Module: U:\extras\lib\db-4.5.lib(hash_stat.obj)
0001:000ca8e0  ___ham_stat
0001:000cb5e0  ___ham_traverse
0001:000cae10  ___ham_stat_print
0001:000cba20  ___ham_print_cursor
Module: U:\extras\lib\db-4.5.lib(qam_stat.obj)
0001:000cbb80  ___qam_stat
0001:000cc3b0  ___qam_stat_print
Module: U:\extras\lib\db-4.5.lib(hash_upgrade.obj)
0001:000cc5e0  ___ham_30_hashmeta
0001:000cc760  ___ham_31_hashmeta
0001:000cc810  ___ham_31_hash
0001:000cc900  ___ham_30_sizefix
Module: U:\extras\lib\db-4.5.lib(bt_upgrade.obj)
0001:000cc9f0  ___bam_31_btreemeta
0001:000cca80  ___bam_30_btreemeta
0001:000ccb00  ___bam_31_lbtree
Module: U:\extras\lib\db-4.5.lib(qam_upgrade.obj)
0001:000ccc70  ___qam_31_qammeta
0001:000cccf0  ___qam_32_qammeta
Module: U:\extras\lib\db-4.5.lib(qam_verify.obj)
0001:000cce50  ___qam_vrfy_meta
0001:000cd3e0  ___qam_vrfy_data
0001:000cd620  ___qam_vrfy_structure
0001:000cd7b0  ___qam_vrfy_walkqueue
0001:000cdb90  ___qam_salvage
Module: U:\extras\lib\db-4.5.lib(hash_verify.obj)
0001:000cdf90  ___ham_vrfy_meta
0001:000ce3a0  ___ham_vrfy
0001:000cec50  ___ham_vrfy_structure
0001:000cf6d0  ___ham_vrfy_hashing
0001:000cf840  ___ham_salvage
0001:000cfd70  ___ham_meta2pgset
Module: U:\extras\lib\db-4.5.lib(bt_verify.obj)
0001:000d0160  ___bam_vrfy_meta
0001:000d0670  ___ram_vrfy_leaf
0001:000d08f0  ___bam_vrfy
0001:000d1bb0  ___bam_vrfy_itemorder
0001:000d23a0  ___bam_vrfy_structure
0001:000d2c00  ___bam_vrfy_subtree
0001:000d3f10  ___bam_salvage
0001:000d4560  ___bam_salvage_walkdupint
0001:000d46d0  ___bam_meta2pgset
Module: U:\extras\lib\db-4.5.lib(db_ovfl_vrfy.obj)
0001:000d4a40  ___db_vrfy_overflow
0001:000d4d20  ___db_vrfy_ovfl_structure
0001:000d5030  ___db_safe_goff
Module: U:\extras\lib\db-4.5.lib(db_log2.obj)
0001:000d5280  ___db_log2
Module: U:\extras\lib\db-4.5.lib(xa.obj)
0001:000d52b0* _db_xa_switch
0001:000d59e0  ___xa_get_txn
Module: U:\extras\lib\db-4.5.lib(rep_auto.obj)
0001:000d5fb0  ___rep_fileinfo_buf
0001:000d6120  ___rep_fileinfo_read
0001:000d61d0  ___rep_update_buf
0001:000d6250  ___rep_update_read
Module: U:\extras\lib\db-4.5.lib(db_meta.obj)
0001:000d62e0  ___db_new
0001:000d7970  ___db_lget
0001:000d7d80  ___db_lput
0001:000d6800  ___db_free
0001:000d6f30  ___db_freelist_pos
0001:000d6f80  ___db_pg_truncate
0001:000d7160  ___db_free_truncate
Module: U:\extras\lib\db-4.5.lib(crdel_rec.obj)
0001:000d7ef0  ___crdel_metasub_recover
0001:000d8240  ___crdel_inmem_create_recover
0001:000d8590  ___crdel_inmem_rename_recover
0001:000d8690  ___crdel_inmem_remove_recover
Module: U:\extras\lib\db-4.5.lib(dbreg_rec.obj)
0001:000d8780  ___dbreg_register_recover
Module: U:\extras\lib\db-4.5.lib(fop_rec.obj)
0001:000d8f90  ___fop_create_recover
0001:000d90e0  ___fop_remove_recover
0001:000d91e0  ___fop_rename_recover
0001:000d96c0  ___fop_file_remove_recover
0001:000d99e0  ___fop_write_recover
Module: U:\extras\lib\db-4.5.lib(qam_rec.obj)
0001:000d9ad0  ___qam_incfirst_recover
0001:000da060  ___qam_mvptr_recover
0001:000da610  ___qam_del_recover
0001:000dac00  ___qam_delext_recover
0001:000db1b0  ___qam_add_recover
Module: U:\extras\lib\db-4.5.lib(db_dup.obj)
0001:000db820  ___db_ditem
0001:000dba10  ___db_pitem
Module: U:\extras\lib\db-4.5.lib(hash_page.obj)
0001:000dbca0  ___ham_item
0001:000df0b0  ___ham_get_cpage
0001:000df260  ___ham_next_cpage
0001:000dbef0  ___ham_item_prev
0001:000dc110  ___ham_item_next
0001:000dc300  ___ham_del_pair
0001:000df390  ___ham_dpair
0001:000dce00  ___ham_replpair
0001:000de520  ___ham_add_el
0001:000dd590  ___ham_onpage_replace
0001:000dd8c0  ___ham_split_page
0001:000def40  ___ham_add_ovflpage
0001:000dedf0  ___ham_copy_item
0001:000df2f0  ___ham_lock_bucket
0001:000df9e0  ___ham_item_reset
0001:000dfac0  ___ham_item_init
0001:000dfb60  ___ham_item_last
0001:000dfbf0  ___ham_item_first
0001:000dfc80  ___ham_putitem
0001:000dfdf0  ___ham_reputpair
Module: U:\extras\lib\db-4.5.lib(hash_meta.obj)
0001:000dffb0  ___ham_get_meta
0001:000e0070  ___ham_release_meta
0001:000e00e0  ___ham_dirty_meta
Module: U:\extras\lib\db-4.5.lib(mp_mvcc.obj)
0001:000e0170  ___memp_bucket_reorder
0001:000e06a0  ___memp_skip_curadj
0001:000e0850  ___memp_bh_freeze
0001:000e1470  ___memp_bh_thaw
0001:000e2530  ___memp_bh_priority
0001:000e25d0  ___memp_bh_settxn
Module: U:\extras\lib\db-4.5.lib(bt_split.obj)
0001:000e2690  ___bam_split
0001:000e3c20  ___bam_pinsert
0001:000e4b70  ___bam_copy
Module: U:\extras\lib\db-4.5.lib(bt_rsearch.obj)
0001:000e4ea0  ___bam_rsearch
0001:000e5580  ___bam_adjust
0001:000e5760  ___bam_total
0001:000e5960  ___bam_nrecs
Module: U:\extras\lib\db-4.5.lib(bt_delete.obj)
0001:000e5a60  ___bam_ditem
0001:000e5cb0  ___bam_adjindx
0001:000e5e10  ___bam_dpages
0001:000e6bb0  ___bam_pupdate
0001:000e67d0  ___bam_relink
Module: U:\extras\lib\db-4.5.lib(bt_curadj.obj)
0001:000e6cc0  ___bam_ca_delete
0001:000e6ea0  ___ram_ca_delete
0001:000e7030  ___bam_ca_di
0001:000e72f0  ___bam_ca_dup
0001:000e7660  ___bam_ca_undodup
0001:000e7870  ___bam_ca_rsplit
0001:000e7b00  ___bam_ca_split
0001:000e7de0  ___bam_ca_undosplit
Module: U:\extras\lib\db-4.5.lib(bt_put.obj)
0001:000e8080  ___bam_iitem
0001:000e8fc0  ___bam_ritem
Module: U:\extras\lib\db-4.5.lib(rijndael-api-fst.obj)
0001:000e98f0  ___db_makeKey
0001:000e99d0  ___db_blockEncrypt
0001:000e9be0* ___db_padEncrypt
0001:000e9e10  ___db_blockDecrypt
0001:000ea070* ___db_padDecrypt
0001:000ea330  ___db_cipherInit
Module: U:\extras\lib\db-4.5.lib(mt19937db.obj)
0001:000ea390  ___db_generate_iv
Module: U:\extras\lib\db-4.5.lib(os_mkdir.obj)
0001:000ea660  ___os_mkdir
Module: U:\extras\lib\db-4.5.lib(bt_search.obj)
0001:000ea750  ___bam_get_root
0001:000ebbf0  ___bam_stkgrow
0001:000eaad0  ___bam_search
0001:000ebad0  ___bam_stkrel
Module: U:\extras\lib\db-4.5.lib(db_reclaim.obj)
0001:000ebcd0  ___db_truncate_callback
0001:000ec330  ___db_traverse_big
0001:000ec400  ___db_reclaim_callback
Module: U:\extras\lib\db-4.5.lib(db_overflow.obj)
0001:000ec450  ___db_goff
0001:000ec6f0  ___db_poff
0001:000ec9b0  ___db_doff
0001:000ecca0  ___db_moff
0001:000ecec0  ___db_ovref
Module: U:\extras\lib\db-4.5.lib(hash_dup.obj)
0001:000ed000  ___ham_add_dup
0001:000ed6f0  ___ham_dup_convert
0001:000ede20  ___ham_make_dup
0001:000eeb60  ___ham_dsearch
Module: U:\extras\lib\db-4.5.lib(db_upg_opd.obj)
0001:000ef060  ___db_31_offdup
Module: U:\extras\lib\db-4.5.lib(xa_map.obj)
0001:000efba0  ___db_rmid_to_env
0001:000efc50  ___db_xid_to_txn
0001:000efc80  ___db_map_rmid
0001:000efcc0  ___db_unmap_rmid
0001:000efd30  ___db_map_xid
0001:000efdd0  ___db_unmap_xid
Module: U:\extras\lib\db-4.5.lib(rijndael-alg-fst.obj)
0001:000f2640  ___db_rijndaelKeySetupEnc
0001:000f2990  ___db_rijndaelKeySetupDec
0001:000f2bc0  ___db_rijndaelEncrypt
0001:000f30a0  ___db_rijndaelDecrypt


                        +----------------------+
                        |   Imported Symbols   |
                        +----------------------+

Symbol                              Module
======                              ======

___libc_ForkRegisterModule          libc064
___init_dll                         libc064
___libc_Back_termDll                libc064
___libc_ForkDeregisterModule        libc064
__atfork_callback                   libc064
__Py_NoneStruct                     python27
_Py_BuildValue                      python27
_PyErr_SetObject                    python27
_PyEval_SaveThread                  python27
_PyEval_RestoreThread               python27
_PyString_FromString                python27
_PyInt_FromLong                     python27
_PyArg_ParseTuple                   python27
_PyDict_SetItemString               python27
_PyErr_Clear                        python27
_PyType_Ready                       python27
_Py_InitModule4                     python27
_PyModule_GetDict                   python27
_PyErr_NewException                 python27
_PyExc_KeyError                     python27
_PyRun_StringFlags                  python27
_PyDict_GetItemString               python27
_PyDict_DelItemString               python27
_PyCObject_FromVoidPtr              python27
_PyErr_Occurred                     python27
_PyErr_Print                        python27
_Py_FatalError                      python27
_PyErr_WriteUnraisable              python27
_PyExc_RuntimeWarning               python27
_PyErr_WarnEx                       python27
_PyExc_TypeError                    python27
_PyErr_Format                       python27
_PyString_FromStringAndSize         python27
_PyGILState_Ensure                  python27
_PyEval_CallObjectWithKeywords      python27
_PyGILState_Release                 python27
_PyArg_Parse                        python27
_PyErr_SetString                    python27
__PyObject_New                      python27
_PyTuple_Pack                       python27
_PyString_AsStringAndSize           python27
_PyInt_AsLong                       python27
_PyExc_MemoryError                  python27
_PyObject_ClearWeakRefs             python27
_PyObject_Free                      python27
_PyArg_ParseTupleAndKeywords        python27
_PyDict_New                         python27
_PyDict_SetItem                     python27
_PyCallable_Check                   python27
_PyEval_InitThreads                 python27
_PyBool_FromLong                    python27
_PyList_New                         python27
_PyTuple_New                        python27
_PyTuple_SetItem                    python27
_PyList_Append                      python27
_PyErr_NoMemory                     python27
_PyLong_FromUnsignedLong            python27
_PyExc_RuntimeError                 python27
_PySequence_Check                   python27
_PyObject_Size                      python27
_PySequence_GetItem                 python27
_PyLong_FromLongLong                python27
__Py_ZeroStruct                     python27
__Py_TrueStruct                     python27
_PyExc_ValueError                   python27
_PyArg_UnpackTuple                  python27
__CRT_init                          libc064
__CRT_term                          libc064
__std_free                          libc064
__std_malloc                        libc064
__std_memcpy                        libc064
___stderrp                          libc064
___stdoutp                          libc064
__std_strncat                       libc064
__std_fopen                         libc064
__std_fclose                        libc064
___ctordtorTerm1                    libc064
___ctordtorInit1                    libc064
___libc_GLocaleCtype                libc064
_strsep                             libc064
__std_strlen                        libc064
__std_strchr                        libc064
__std_strcat                        libc064
__std_strerror                      libc064
__std_snprintf                      libc064
__std_vsnprintf                     libc064
__errno                             libc064
__std_vfprintf                      libc064
__std_fputc                         libc064
__std_fflush                        libc064
__std_fwrite                        libc064
__std_fputs                         libc064
__std_fprintf                       libc064
__std_memset                        libc064
___deregister_frame                 gcc446
___register_frame_table             gcc446
__std_time                          libc064
__std_strncpy                       libc064
__std_atol                          libc064
__std_realloc                       libc064
__std_fgets                         libc064
__std_stricmp                       libc064
__std_getuid                        libc064
__std_getenv                        libc064
__std_strcpy                        libc064
__std_qsort                         libc064
__std_stat                          libc064
__std_fstat                         libc064
__std_getpid                        libc064
__std_fchmod                        libc064
__std_strcmp                        libc064
__std_localtime                     libc064
__std_strftime                      libc064
__std_getcwd                        libc064
__std_select                        libc064
__std_open                          libc064
__std_fcntl                         libc064
__std_close                         libc064
__std_rand                          libc064
__std_srand                         libc064
__std_pwrite                        libc064
__std_pread                         libc064
__std_read                          libc064
__std_write                         libc064
__std_opendir                       libc064
__std_readdir                       libc064
__std_closedir                      libc064
__std_unlink                        libc064
__std_sysconf                       libc064
__std_lseek                         libc064
__std_gettimeofday                  libc064
__std_memmove                       libc064
__std_ctime_r                       libc064
__std_fsync                         libc064
__std_strtol                        libc064
__std_strtoul                       libc064
__std_putchar                       libc064
__std_printf                        libc064
__std_fgetc                         libc064
__std_strrchr                       libc064
__std_strncmp                       libc064
__std_rename                        libc064
__std_ftruncate                     libc064
__std_shmget                        libc064
__std_shmctl                        libc064
__std_shmat                         libc064
__std_shmdt                         libc064
__std_mkdir                         libc064
__std_chmod                         libc064


                        +--------------------+
                        |   Libraries Used   |
                        +--------------------+

U:\extras\lib\db-4.5.lib
U:\tmp\ldconv_python2_7_dll_a_ddce4f08029e15d430.lib
U:\usr\local446\lib\gcc\i386-pc-os2-emx\4.4.6\libgcc.lib
U:\tmp\ldconv_libgcc_so_d_a_ddce4f08029e1635d8.lib
U:\usr\lib\libc_alias.lib
U:\usr\local446\lib\libc_dll.lib
U:\usr\lib\libend.lib


                        +-----------------------+
                        |   Linker Statistics   |
                        +-----------------------+

Stack size:  0000 (0.)
Memory size:  000f58e0 (1005792.)
Link time: 00:00.16
